Archive member included because of file (symbol)

c:/winavr-20100110/bin/../lib/gcc/avr/4.3.3/avr4\libgcc.a(_mulsi3.o)
                              main.o (__mulsi3)
c:/winavr-20100110/bin/../lib/gcc/avr/4.3.3/avr4\libgcc.a(_udivmodhi4.o)
                              main.o (__udivmodhi4)
c:/winavr-20100110/bin/../lib/gcc/avr/4.3.3/avr4\libgcc.a(_exit.o)
                              c:/winavr-20100110/bin/../lib/gcc/avr/4.3.3/../../../../avr/lib/avr4/crtm88.o (exit)
c:/winavr-20100110/bin/../lib/gcc/avr/4.3.3/avr4\libgcc.a(_copy_data.o)
                              cc1100.o (__do_copy_data)
c:/winavr-20100110/bin/../lib/gcc/avr/4.3.3/avr4\libgcc.a(_clear_bss.o)
                              cc1100.o (__do_clear_bss)
c:/winavr-20100110/bin/../lib/gcc/avr/4.3.3/../../../../avr/lib/avr4\libc.a(memcmp.o)
                              main.o (memcmp)
c:/winavr-20100110/bin/../lib/gcc/avr/4.3.3/../../../../avr/lib/avr4\libc.a(memset.o)
                              main.o (memset)
c:/winavr-20100110/bin/../lib/gcc/avr/4.3.3/../../../../avr/lib/avr4\libc.a(eerd_block_atmega88.o)
                              main.o (__eerd_block_m88)
c:/winavr-20100110/bin/../lib/gcc/avr/4.3.3/../../../../avr/lib/avr4\libc.a(eerd_byte_atmega88.o)
                              main.o (__eerd_byte_m88)
c:/winavr-20100110/bin/../lib/gcc/avr/4.3.3/../../../../avr/lib/avr4\libc.a(eewr_block_atmega88.o)
                              main.o (__eewr_block_m88)
c:/winavr-20100110/bin/../lib/gcc/avr/4.3.3/../../../../avr/lib/avr4\libc.a(eewr_byte_atmega88.o)
                              c:/winavr-20100110/bin/../lib/gcc/avr/4.3.3/../../../../avr/lib/avr4\libc.a(eewr_block_atmega88.o) (__eewr_r18_m88)

Allocating common symbols
Common symbol       size              file

frq_data            0x1               main.o
tLength             0x1               main.o
uart_data           0x1               main.o
gOpt                0xf               main.o
tSlave              0x4               main.o
pC                  0x2               main.o
gClient             0x49              main.o
pt_reg              0xa               cc1100.o
gLevel              0x1               main.o
tSlave2             0x4               main.o
gTemperature        0x2               main.o
tCtl                0x7               main.o
tTemp               0x1               main.o

Memory Configuration

Name             Origin             Length             Attributes
text             0x00000000         0x00002000         xr
data             0x00800060         0x0000ffa0         rw !x
eeprom           0x00810000         0x00010000         rw !x
fuse             0x00820000         0x00000400         rw !x
lock             0x00830000         0x00000400         rw !x
signature        0x00840000         0x00000400         rw !x
*default*        0x00000000         0xffffffff

Linker script and memory map

Address of section .data set to 0x800100
LOAD c:/winavr-20100110/bin/../lib/gcc/avr/4.3.3/../../../../avr/lib/avr4/crtm88.o
LOAD cc1100.o
LOAD main.o
LOAD spi1.o
LOAD i2c.o
LOAD c:/winavr-20100110/bin/../lib/gcc/avr/4.3.3/avr4\libgcc.a
LOAD c:/winavr-20100110/bin/../lib/gcc/avr/4.3.3/../../../../avr/lib/avr4\libc.a
LOAD c:/winavr-20100110/bin/../lib/gcc/avr/4.3.3/avr4\libgcc.a

.hash
 *(.hash)

.dynsym
 *(.dynsym)

.dynstr
 *(.dynstr)

.gnu.version
 *(.gnu.version)

.gnu.version_d
 *(.gnu.version_d)

.gnu.version_r
 *(.gnu.version_r)

.rel.init
 *(.rel.init)

.rela.init
 *(.rela.init)

.rel.text
 *(.rel.text)
 *(.rel.text.*)
 *(.rel.gnu.linkonce.t*)

.rela.text
 *(.rela.text)
 *(.rela.text.*)
 *(.rela.gnu.linkonce.t*)

.rel.fini
 *(.rel.fini)

.rela.fini
 *(.rela.fini)

.rel.rodata
 *(.rel.rodata)
 *(.rel.rodata.*)
 *(.rel.gnu.linkonce.r*)

.rela.rodata
 *(.rela.rodata)
 *(.rela.rodata.*)
 *(.rela.gnu.linkonce.r*)

.rel.data
 *(.rel.data)
 *(.rel.data.*)
 *(.rel.gnu.linkonce.d*)

.rela.data
 *(.rela.data)
 *(.rela.data.*)
 *(.rela.gnu.linkonce.d*)

.rel.ctors
 *(.rel.ctors)

.rela.ctors
 *(.rela.ctors)

.rel.dtors
 *(.rel.dtors)

.rela.dtors
 *(.rela.dtors)

.rel.got
 *(.rel.got)

.rela.got
 *(.rela.got)

.rel.bss
 *(.rel.bss)

.rela.bss
 *(.rela.bss)

.rel.plt
 *(.rel.plt)

.rela.plt
 *(.rela.plt)

.text           0x00000000     0x14fa
 *(.vectors)
 .vectors       0x00000000       0x34 c:/winavr-20100110/bin/../lib/gcc/avr/4.3.3/../../../../avr/lib/avr4/crtm88.o
                0x00000000                __vectors
                0x00000000                __vector_default
 *(.vectors)
 *(.progmem.gcc*)
 *(.progmem*)
                0x00000034                . = ALIGN (0x2)
                0x00000034                __trampolines_start = .
 *(.trampolines)
 .trampolines   0x00000034        0x0 linker stubs
 *(.trampolines*)
                0x00000034                __trampolines_end = .
 *(.jumptables)
 *(.jumptables*)
 *(.lowtext)
 *(.lowtext*)
                0x00000034                __ctors_start = .
 *(.ctors)
                0x00000034                __ctors_end = .
                0x00000034                __dtors_start = .
 *(.dtors)
                0x00000034                __dtors_end = .
 SORT(*)(.ctors)
 SORT(*)(.dtors)
 *(.init0)
 .init0         0x00000034        0x0 c:/winavr-20100110/bin/../lib/gcc/avr/4.3.3/../../../../avr/lib/avr4/crtm88.o
                0x00000034                __init
 *(.init0)
 *(.init1)
 *(.init1)
 *(.init2)
 .init2         0x00000034        0xc c:/winavr-20100110/bin/../lib/gcc/avr/4.3.3/../../../../avr/lib/avr4/crtm88.o
 *(.init2)
 *(.init3)
 *(.init3)
 *(.init4)
 .init4         0x00000040       0x16 c:/winavr-20100110/bin/../lib/gcc/avr/4.3.3/avr4\libgcc.a(_copy_data.o)
                0x00000040                __do_copy_data
 .init4         0x00000056       0x10 c:/winavr-20100110/bin/../lib/gcc/avr/4.3.3/avr4\libgcc.a(_clear_bss.o)
                0x00000056                __do_clear_bss
 *(.init4)
 *(.init5)
 *(.init5)
 *(.init6)
 *(.init6)
 *(.init7)
 *(.init7)
 *(.init8)
 *(.init8)
 *(.init9)
 .init9         0x00000066        0x4 c:/winavr-20100110/bin/../lib/gcc/avr/4.3.3/../../../../avr/lib/avr4/crtm88.o
 *(.init9)
 *(.text)
 .text          0x0000006a        0x2 c:/winavr-20100110/bin/../lib/gcc/avr/4.3.3/../../../../avr/lib/avr4/crtm88.o
                0x0000006a                __vector_22
                0x0000006a                __vector_24
                0x0000006a                __vector_12
                0x0000006a                __bad_interrupt
                0x0000006a                __vector_6
                0x0000006a                __vector_3
                0x0000006a                __vector_23
                0x0000006a                __vector_25
                0x0000006a                __vector_11
                0x0000006a                __vector_13
                0x0000006a                __vector_17
                0x0000006a                __vector_19
                0x0000006a                __vector_7
                0x0000006a                __vector_5
                0x0000006a                __vector_4
                0x0000006a                __vector_9
                0x0000006a                __vector_2
                0x0000006a                __vector_21
                0x0000006a                __vector_15
                0x0000006a                __vector_8
                0x0000006a                __vector_14
                0x0000006a                __vector_10
                0x0000006a                __vector_16
                0x0000006a                __vector_18
                0x0000006a                __vector_20
 .text          0x0000006c      0x234 cc1100.o
                0x000001ae                cc1100_strobe_cmd
                0x00000080                cc1100_sleep_strobe_cmd
                0x00000150                cc1100_read_status
                0x00000076                cc1100_gdo2_register_callback
                0x00000182                cc1100_fifo_put
                0x00000220                cc1100_init
                0x00000156                cc1100_fifo_get
                0x000000ae                cc1100_write_reg
                0x000001d0                cc1100_cmd_idle
                0x0000021c                cc1100_reinit
                0x000000d0                cc1101_init_reg
                0x00000106                cc1101_8PATABLE_read_reg
                0x00000130                cc1100_read_reg
                0x0000020a                cc1100_cmd_calibrate
                0x0000006c                cc1100_gdo0_register_callback
                0x00000084                cc1101_8PATABLE_write_reg
                0x000000ee                cc1101_rtx_reg_set
 .text          0x000002a0      0xf12 main.o
                0x000002b6                mdelay
                0x00000824                sleep_set
                0x00000868                __vector_1
                0x00000328                putb
                0x00000b88                cc1101_carrier_wave_setup
                0x000006ea                cc1101_carrier_frq_setup
                0x00000d7c                cc1101_tx_carrier
                0x00000656                get_stop_signal
                0x0000046a                led_onoff
                0x00000394                putstr
                0x00000844                set_cur_status
                0x00000370                chr2hex
                0x000009a8                tx_fifo_write
                0x00000318                putc_
                0x00000fbe                slave_oper
                0x0000034a                puthex
                0x00000b80                my_eeprom_read_byte
                0x00000aca                reg_slave_num_serch
                0x00000958                rx_fifo_read
                0x000004d0                inituart
                0x00000eb2                setup_oper
                0x0000073a                temperature_test_disenable
                0x0000059c                get_freq_data
                0x000002f0                sdelay
                0x0000075a                temperature_get
                0x00000e04                slave_fifo_preset
                0x000009de                my_eeprom_read_block
                0x00000446                hexToAsc
                0x0000040a                asc_to_int
                0x0000061c                sig_status
                0x00000906                carrier_test
                0x00000aa0                device_status_setup
                0x000005a8                get_mode_data
                0x000002a0                udelay
                0x00000f72                setup_main
                0x0000035e                putchr2hex
                0x00000438                hex_to_asc
                0x000008b2                cc1101_tx_carrier_test
                0x00001032                slave_main
                0x000003c2                asc_to_hex
                0x000009d8                get_cur_status
                0x00000d02                cc1101_tx
                0x00000cb2                cc1101_rx
                0x00000414                AscToInt
                0x000004f2                hw_setup
                0x00000748                temperature_test_enable
                0x000003e6                AscToHex
                0x00001110                main
                0x00000522                ad_get_val
                0x00000682                get_emg_signal
                0x000009e6                check_env
                0x000005fe                add_batt_low
                0x00000796                rtc_set_next_alarm
                0x0000067e                power_off
                0x0000062a                carrier_no_sense
                0x0000048e                led_flasher
                0x0000084c                rtc_alarm_disenable
                0x00000dd0                temperature_carrier_test
                0x000006aa                hex_change_level
                0x000005b0                level_change_hex
                0x000005f2                init_voltcomparator
                0x00000624                carrier_sense
                0x00000630                my_memcmp
 .text          0x000011b2       0xd2 spi1.o
                0x00001210                spi1_read
                0x00001246                spi1_read_somi
                0x000011c4                spi1_write_single
                0x0000126e                spi_signalpin_opendrain_nonactive
                0x0000123e                spi1_deselect
                0x000011e8                spi1_write
                0x00001252                spi_signalpin_opendrain_active
                0x000011d6                spi1_read_single
                0x000011b2                spi1_init
                0x00001236                spi1_select
 .text          0x00001284      0x186 i2c.o
                0x00001308                i2c_read_nak
                0x00001398                rtc_1byte_data_read
                0x0000133c                i2c_write
                0x000012a0                i2c_wait_int_clear
                0x00001322                i2c_read_ack
                0x000012cc                i2c_start
                0x00001356                rtc_3byte_data_read
                0x00001290                i2c_stop
                0x000013c8                rtc_1byte_data_write
                0x000012be                i2c_error
                0x00001284                i2c_init
 .text          0x0000140a        0x0 c:/winavr-20100110/bin/../lib/gcc/avr/4.3.3/avr4\libgcc.a(_mulsi3.o)
 .text          0x0000140a        0x0 c:/winavr-20100110/bin/../lib/gcc/avr/4.3.3/avr4\libgcc.a(_udivmodhi4.o)
 .text          0x0000140a        0x0 c:/winavr-20100110/bin/../lib/gcc/avr/4.3.3/avr4\libgcc.a(_exit.o)
 .text          0x0000140a        0x0 c:/winavr-20100110/bin/../lib/gcc/avr/4.3.3/avr4\libgcc.a(_copy_data.o)
 .text          0x0000140a        0x0 c:/winavr-20100110/bin/../lib/gcc/avr/4.3.3/avr4\libgcc.a(_clear_bss.o)
 .text          0x0000140a        0x0 c:/winavr-20100110/bin/../lib/gcc/avr/4.3.3/../../../../avr/lib/avr4\libc.a(memcmp.o)
 .text          0x0000140a        0x0 c:/winavr-20100110/bin/../lib/gcc/avr/4.3.3/../../../../avr/lib/avr4\libc.a(memset.o)
 .text          0x0000140a        0x0 c:/winavr-20100110/bin/../lib/gcc/avr/4.3.3/../../../../avr/lib/avr4\libc.a(eerd_block_atmega88.o)
 .text          0x0000140a        0x0 c:/winavr-20100110/bin/../lib/gcc/avr/4.3.3/../../../../avr/lib/avr4\libc.a(eerd_byte_atmega88.o)
 .text          0x0000140a        0x0 c:/winavr-20100110/bin/../lib/gcc/avr/4.3.3/../../../../avr/lib/avr4\libc.a(eewr_block_atmega88.o)
 .text          0x0000140a        0x0 c:/winavr-20100110/bin/../lib/gcc/avr/4.3.3/../../../../avr/lib/avr4\libc.a(eewr_byte_atmega88.o)
                0x0000140a                . = ALIGN (0x2)
 *(.text.*)
 .text.libgcc   0x0000140a       0x3e c:/winavr-20100110/bin/../lib/gcc/avr/4.3.3/avr4\libgcc.a(_mulsi3.o)
                0x0000140a                __mulsi3
 .text.libgcc   0x00001448       0x28 c:/winavr-20100110/bin/../lib/gcc/avr/4.3.3/avr4\libgcc.a(_udivmodhi4.o)
                0x00001448                __udivmodhi4
 .text.libgcc   0x00001470        0x0 c:/winavr-20100110/bin/../lib/gcc/avr/4.3.3/avr4\libgcc.a(_exit.o)
 .text.libgcc   0x00001470        0x0 c:/winavr-20100110/bin/../lib/gcc/avr/4.3.3/avr4\libgcc.a(_copy_data.o)
 .text.libgcc   0x00001470        0x0 c:/winavr-20100110/bin/../lib/gcc/avr/4.3.3/avr4\libgcc.a(_clear_bss.o)
 .text.avr-libc
                0x00001470       0x1a c:/winavr-20100110/bin/../lib/gcc/avr/4.3.3/../../../../avr/lib/avr4\libc.a(memcmp.o)
                0x00001470                memcmp
 .text.avr-libc
                0x0000148a        0xe c:/winavr-20100110/bin/../lib/gcc/avr/4.3.3/../../../../avr/lib/avr4\libc.a(memset.o)
                0x0000148a                memset
 .text.avr-libc
                0x00001498       0x20 c:/winavr-20100110/bin/../lib/gcc/avr/4.3.3/../../../../avr/lib/avr4\libc.a(eerd_block_atmega88.o)
                0x0000149c                __eerd_blraw_m88
                0x00001498                __eerd_block_m88
 .text.avr-libc
                0x000014b8       0x10 c:/winavr-20100110/bin/../lib/gcc/avr/4.3.3/../../../../avr/lib/avr4\libc.a(eerd_byte_atmega88.o)
                0x000014b8                __eerd_byte_m88
 .text.avr-libc
                0x000014c8       0x12 c:/winavr-20100110/bin/../lib/gcc/avr/4.3.3/../../../../avr/lib/avr4\libc.a(eewr_block_atmega88.o)
                0x000014c8                __eewr_block_m88
 .text.avr-libc
                0x000014da       0x1c c:/winavr-20100110/bin/../lib/gcc/avr/4.3.3/../../../../avr/lib/avr4\libc.a(eewr_byte_atmega88.o)
                0x000014dc                __eewr_r18_m88
                0x000014da                __eewr_byte_m88
                0x000014f6                . = ALIGN (0x2)
 *(.fini9)
 .fini9         0x000014f6        0x0 c:/winavr-20100110/bin/../lib/gcc/avr/4.3.3/avr4\libgcc.a(_exit.o)
                0x000014f6                exit
                0x000014f6                _exit
 *(.fini9)
 *(.fini8)
 *(.fini8)
 *(.fini7)
 *(.fini7)
 *(.fini6)
 *(.fini6)
 *(.fini5)
 *(.fini5)
 *(.fini4)
 *(.fini4)
 *(.fini3)
 *(.fini3)
 *(.fini2)
 *(.fini2)
 *(.fini1)
 *(.fini1)
 *(.fini0)
 .fini0         0x000014f6        0x4 c:/winavr-20100110/bin/../lib/gcc/avr/4.3.3/avr4\libgcc.a(_exit.o)
 *(.fini0)
                0x000014fa                _etext = .

.data           0x00800100       0x88 load address 0x000014fa
                0x00800100                PROVIDE (__data_start, .)
 *(.data)
 .data          0x00800100        0x0 c:/winavr-20100110/bin/../lib/gcc/avr/4.3.3/../../../../avr/lib/avr4/crtm88.o
 .data          0x00800100       0x1c cc1100.o
                0x00800100                pt_data
                0x00800108                init_all
 .data          0x0080011c       0x6b main.o
                0x00800136                reg_next_sch_alarm
                0x00800128                reg_net_alarm
                0x0080014f                level_offset
                0x00800148                day_cnt
                0x0080016b                default_offset
                0x0080014c                fix_id_mel
                0x0080011c                time_set
 .data          0x00800187        0x0 spi1.o
 .data          0x00800187        0x0 i2c.o
 .data          0x00800187        0x0 c:/winavr-20100110/bin/../lib/gcc/avr/4.3.3/avr4\libgcc.a(_mulsi3.o)
 .data          0x00800187        0x0 c:/winavr-20100110/bin/../lib/gcc/avr/4.3.3/avr4\libgcc.a(_udivmodhi4.o)
 .data          0x00800187        0x0 c:/winavr-20100110/bin/../lib/gcc/avr/4.3.3/avr4\libgcc.a(_exit.o)
 .data          0x00800187        0x0 c:/winavr-20100110/bin/../lib/gcc/avr/4.3.3/avr4\libgcc.a(_copy_data.o)
 .data          0x00800187        0x0 c:/winavr-20100110/bin/../lib/gcc/avr/4.3.3/avr4\libgcc.a(_clear_bss.o)
 .data          0x00800187        0x0 c:/winavr-20100110/bin/../lib/gcc/avr/4.3.3/../../../../avr/lib/avr4\libc.a(memcmp.o)
 .data          0x00800187        0x0 c:/winavr-20100110/bin/../lib/gcc/avr/4.3.3/../../../../avr/lib/avr4\libc.a(memset.o)
 .data          0x00800187        0x0 c:/winavr-20100110/bin/../lib/gcc/avr/4.3.3/../../../../avr/lib/avr4\libc.a(eerd_block_atmega88.o)
 .data          0x00800187        0x0 c:/winavr-20100110/bin/../lib/gcc/avr/4.3.3/../../../../avr/lib/avr4\libc.a(eerd_byte_atmega88.o)
 .data          0x00800187        0x0 c:/winavr-20100110/bin/../lib/gcc/avr/4.3.3/../../../../avr/lib/avr4\libc.a(eewr_block_atmega88.o)
 .data          0x00800187        0x0 c:/winavr-20100110/bin/../lib/gcc/avr/4.3.3/../../../../avr/lib/avr4\libc.a(eewr_byte_atmega88.o)
 *(.data*)
 *(.rodata)
 *(.rodata*)
 *(.gnu.linkonce.d*)
                0x00800188                . = ALIGN (0x2)
 *fill*         0x00800187        0x1 00
                0x00800188                _edata = .
                0x00800188                PROVIDE (__data_end, .)

.bss            0x00800188       0x87
                0x00800188                PROVIDE (__bss_start, .)
 *(.bss)
 .bss           0x00800188        0x0 c:/winavr-20100110/bin/../lib/gcc/avr/4.3.3/../../../../avr/lib/avr4/crtm88.o
 .bss           0x00800188        0x4 cc1100.o
 .bss           0x0080018c        0x7 main.o
                0x00800190                gRecvRssi
                0x00800191                gRecvLqi
                0x0080018e                setup_mode
                0x0080018c                get_user0_data
                0x00800192                gStatus
                0x0080018d                emg_status
                0x0080018f                gslave_master_ctl
 .bss           0x00800193        0x1 spi1.o
                0x00800193                spi_active
 .bss           0x00800194        0x1 i2c.o
                0x00800194                i2c_error_flag
 .bss           0x00800195        0x0 c:/winavr-20100110/bin/../lib/gcc/avr/4.3.3/avr4\libgcc.a(_mulsi3.o)
 .bss           0x00800195        0x0 c:/winavr-20100110/bin/../lib/gcc/avr/4.3.3/avr4\libgcc.a(_udivmodhi4.o)
 .bss           0x00800195        0x0 c:/winavr-20100110/bin/../lib/gcc/avr/4.3.3/avr4\libgcc.a(_exit.o)
 .bss           0x00800195        0x0 c:/winavr-20100110/bin/../lib/gcc/avr/4.3.3/avr4\libgcc.a(_copy_data.o)
 .bss           0x00800195        0x0 c:/winavr-20100110/bin/../lib/gcc/avr/4.3.3/avr4\libgcc.a(_clear_bss.o)
 .bss           0x00800195        0x0 c:/winavr-20100110/bin/../lib/gcc/avr/4.3.3/../../../../avr/lib/avr4\libc.a(memcmp.o)
 .bss           0x00800195        0x0 c:/winavr-20100110/bin/../lib/gcc/avr/4.3.3/../../../../avr/lib/avr4\libc.a(memset.o)
 .bss           0x00800195        0x0 c:/winavr-20100110/bin/../lib/gcc/avr/4.3.3/../../../../avr/lib/avr4\libc.a(eerd_block_atmega88.o)
 .bss           0x00800195        0x0 c:/winavr-20100110/bin/../lib/gcc/avr/4.3.3/../../../../avr/lib/avr4\libc.a(eerd_byte_atmega88.o)
 .bss           0x00800195        0x0 c:/winavr-20100110/bin/../lib/gcc/avr/4.3.3/../../../../avr/lib/avr4\libc.a(eewr_block_atmega88.o)
 .bss           0x00800195        0x0 c:/winavr-20100110/bin/../lib/gcc/avr/4.3.3/../../../../avr/lib/avr4\libc.a(eewr_byte_atmega88.o)
 *(.bss*)
 *(COMMON)
 COMMON         0x00800195        0xa cc1100.o
                0x00800195                pt_reg
 COMMON         0x0080019f       0x70 main.o
                0x0080019f                frq_data
                0x008001a0                tLength
                0x008001a1                uart_data
                0x008001a2                gOpt
                0x008001b1                tSlave
                0x008001b5                pC
                0x008001b7                gClient
                0x00800200                gLevel
                0x00800201                tSlave2
                0x00800205                gTemperature
                0x00800207                tCtl
                0x0080020e                tTemp
                0x0080020f                PROVIDE (__bss_end, .)
                0x000014fa                __data_load_start = LOADADDR (.data)
                0x00001582                __data_load_end = (__data_load_start + SIZEOF (.data))

.noinit         0x0080020f        0x0
                0x0080020f                PROVIDE (__noinit_start, .)
 *(.noinit*)
                0x0080020f                PROVIDE (__noinit_end, .)
                0x0080020f                _end = .
                0x0080020f                PROVIDE (__heap_start, .)

.eeprom         0x00810000      0x1b3
 *(.eeprom*)
 .eeprom        0x00810000      0x1b3 main.o
                0x00810007                greg_slave
                0x00810197                eprom_level
                0x00810000                gctl_data
                0x008101b3                __eeprom_end = .

.fuse
 *(.fuse)
 *(.lfuse)
 *(.hfuse)
 *(.efuse)

.lock
 *(.lock*)

.signature
 *(.signature*)

.stab
 *(.stab)

.stabstr
 *(.stabstr)

.stab.excl
 *(.stab.excl)

.stab.exclstr
 *(.stab.exclstr)

.stab.index
 *(.stab.index)

.stab.indexstr
 *(.stab.indexstr)

.comment
 *(.comment)

.debug
 *(.debug)

.line
 *(.line)

.debug_srcinfo
 *(.debug_srcinfo)

.debug_sfnames
 *(.debug_sfnames)

.debug_aranges  0x00000000       0x80
 *(.debug_aranges)
 .debug_aranges
                0x00000000       0x20 cc1100.o
 .debug_aranges
                0x00000020       0x20 main.o
 .debug_aranges
                0x00000040       0x20 spi1.o
 .debug_aranges
                0x00000060       0x20 i2c.o

.debug_pubnames
                0x00000000      0x9a8
 *(.debug_pubnames)
 .debug_pubnames
                0x00000000      0x1c9 cc1100.o
 .debug_pubnames
                0x000001c9      0x5ff main.o
 .debug_pubnames
                0x000007c8       0xf5 spi1.o
 .debug_pubnames
                0x000008bd       0xeb i2c.o

.debug_info     0x00000000     0x2328
 *(.debug_info)
 .debug_info    0x00000000      0x44c cc1100.o
 .debug_info    0x0000044c     0x19ec main.o
 .debug_info    0x00001e38      0x29c spi1.o
 .debug_info    0x000020d4      0x254 i2c.o
 *(.gnu.linkonce.wi.*)

.debug_abbrev   0x00000000      0x8c8
 *(.debug_abbrev)
 .debug_abbrev  0x00000000      0x1a4 cc1100.o
 .debug_abbrev  0x000001a4      0x47f main.o
 .debug_abbrev  0x00000623      0x186 spi1.o
 .debug_abbrev  0x000007a9      0x11f i2c.o

.debug_line     0x00000000     0x1c1c
 *(.debug_line)
 .debug_line    0x00000000      0x3a9 cc1100.o
 .debug_line    0x000003a9     0x1360 main.o
 .debug_line    0x00001709      0x242 spi1.o
 .debug_line    0x0000194b      0x2d1 i2c.o

.debug_frame    0x00000000      0x690
 *(.debug_frame)
 .debug_frame   0x00000000      0x120 cc1100.o
 .debug_frame   0x00000120      0x400 main.o
 .debug_frame   0x00000520       0xb0 spi1.o
 .debug_frame   0x000005d0       0xc0 i2c.o

.debug_str      0x00000000      0xbfb
 *(.debug_str)
 .debug_str     0x00000000      0x283 cc1100.o
                                0x2cd (size before relaxing)
 .debug_str     0x00000283      0x7ef main.o
                                0x986 (size before relaxing)
 .debug_str     0x00000a72       0xcc spi1.o
                                0x1e3 (size before relaxing)
 .debug_str     0x00000b3e       0xbd i2c.o
                                0x1a4 (size before relaxing)

.debug_loc      0x00000000      0xc9b
 *(.debug_loc)
 .debug_loc     0x00000000      0x182 cc1100.o
 .debug_loc     0x00000182      0x95a main.o
 .debug_loc     0x00000adc       0xa7 spi1.o
 .debug_loc     0x00000b83      0x118 i2c.o

.debug_macinfo
 *(.debug_macinfo)
OUTPUT(CC1101driver.elf elf32-avr)
LOAD linker stubs

.debug_ranges   0x00000000       0x18
 .debug_ranges  0x00000000       0x18 main.o
